:020000040000FA
:1000000061EF2BF01200FFFFFFFFFFFFFFFFFFFF7D
:10001000FFFFFFFFFFFFFFFFFFFFFFFFFFFFFFFFF0
:10002000FFFFFFFFFFFFFFFFFFFFFFFFFFFFFFFFE0
:10003000FFFFFFFFFFFFFFFFFFFFFFFFFFFFFFFFD0
:10004000FFFFFFFFFFFFFFFFFFFFFFFFFFFFFFFFC0
:1008000061EF2BF01200FFFF1200FFFFFFFFFFFF61
:10081000FFFFFFFFFFFFFFFF1200FFFFFFFFFFFFD4
:10082000FFFFFFFFFFFFFFFFFFFF01003257000048
:10083000CA01000025000000D9CFE6FFE1CFD9FFB3
:10084000E6520101CC6B7F0ECD6FCE69C70ECF6F24
:10085000926893689468DF6ADFCF10F0050EE76E48
:100860001018E8AE02D0E73402D0E750105C01E384
:100870007BD0DFCFE9FFEA6AE9BEEA68040ED890D0
:10088000E936EA36E806FBE1410EE926010EEA22E6
:10089000EF6ADFCFE9FFEA6AE9BEEA68040ED890A2
:1008A000E936EA36E806FBE1410EE926010EEA22C6
:1008B000EE52EF6ADFCFE9FFEA6AE9BEEA68040EAA
:1008C000D890E936EA36E806FBE1410EE926010E4A
:1008D000EA22020EE926000EEA22EF6ADFCFE9FFE4
:1008E000EA6AE9BEEA68040ED890E936EA36E80614
:1008F000FBE1410EE926010EEA22030EE926000E75
:10090000EA22010EEF6EDFCFE9FFEA6AE9BEEA688C
:10091000040ED890E936EA36E806FBE1410EE926F6
:10092000010EEA22040EE926000EEA22EE6AED6AC2
:10093000DFCFE9FFEA6AE9BEEA68040ED890E9363B
:10094000EA36E806FBE1410EE926010EEA22060E30
:10095000E926000EEA22EE6AED6ADFCFE6FFA2EC9E
:1009600013F0E552DF2A78D7DF6ADFCF10F0050EEB
:10097000E76E1018E8AE02D0E73402D0E750105C02
:100980005AE2DFCFE9FFEA6AE9BEEA68050EEA0249
:10099000F3CFEAFFE902F3CFE9FFF450EA26910E24
:1009A000E926010EEA22EF6ADFCFE9FFEA6AE9BE33
:1009B000EA68050EEA02F3CFEAFFE902F3CFE9FFA6
:1009C000F450EA26910EE926010EEA22EE52EF6A71
:1009D000DFCFE9FFEA6AE9BEEA68050EEA02F3CF73
:1009E000EAFFE902F3CFE9FFF450EA26910EE92687
:1009F000010EEA22020EE926000EEA22010EEF6E37
:100A0000DFCFE9FFEA6AE9BEEA68050EEA02F3CF42
:100A1000EAFFE902F3CFE9FFF450EA26910EE92656
:100A2000010EEA22030EE926000EEA22010EEE6E06
:100A3000ED6ADF2A9AD7E552E552E7CFD9FF1200D7
:100A4000060E0101F95D05E36D50020B01E0120095
:100A500001D81200D9CFE6FFE1CFD9FF050EE1267C
:100A6000400EE66E010EE66E010EE66E30EC27F0EB
:100A7000E552E552E552000901E1E5D00101006BC4
:100A800001010151FF0A01E1A5D0960A01E19FD0C1
:100A9000010A01E199D00D0A01E193D0010A01E1B7
:100AA0008DD0070A01E184D0010A01E17BD0030A5D
:100AB00073E0010A6BE03C0A63E0030A5BE0010AB1
:100AC00053E0030A4BE0070A46E0020A41E00F0A3E
:100AD0003CE0010A37E0030A32E0330A2DE0010A64
:100AE00028E0340A23E0070A1EE00D0A19E00B0A89
:100AF00015E0030A11E0010A0DE0500A01E08CD074
:100B00000101090E036F0101020E046F0101040EC1
:100B1000006F88D0F1D886D086D984D07CDA82D094
:100B2000D1EC09F07FD0C4EC0BF07CD050EC0DF090
:100B300079D058EC0EF076D0AEEC0EF073D00AEC13
:100B400010F070D00AEC10F06DD04CEC11F06AD0BF
:100B5000E8EC11F067D084EC12F064D0010EE66E80
:100B6000B6EC15F0E5525ED0020EE66EB6EC15F06E
:100B7000E55258D0030EE66EB6EC15F0E55252D0B1
:100B8000040EE66EB6EC15F0E5524CD0010EE66EA2
:100B900042EC1BF0E55246D0020EE66E42EC1BF032
:100BA000E55240D0030EE66E42EC1BF0E5523AD01F
:100BB000040EE66E42EC1BF0E55234D05EEC1EF003
:100BC00031D09AEC1EF02ED037EC21F02BD088ECEF
:100BD00021F028D06D96010EDB6A020EDB6A010E51
:100BE000DB06DBCF10F0020E01E2DB06DBCF11F0FB
:100BF0001050111001E0F3D7FA0EE66EE66A36ECFB
:100C000022F0E552E552FA0EE66EE66A36EC22F084
:100C1000E552E552FF0006D0010101690101100E05
:100C2000006F00D0010100510EE004010CBF0BD099
:100C300000C1E6FF010EE66E010EE66EF6EC26F050
:100C4000E552E552E5520101D70502E1F6EC0AF062
:100C50000101520505E1010EE66E06EC1AF0E552BF
:100C60000101620505E1020EE66E06EC1AF0E5529E
:100C70000101720505E1030EE66E06EC1AF0E5527D
:100C80000101820505E1040EE66E06EC1AF0E5525C
:100C90000101965105E0010EE66E96EC1DF0E5525D
:100CA00001019B5105E0020EE66E96EC1DF0E55247
:100CB0000101A05105E0030EE66E96EC1DF0E55231
:100CC0000101A55105E0040EE66E96EC1DF0E5521B
:100CD0000101D90502E1D6EC1EF00101E30502E1B4
:100CE00041EC20F0050EE15C02E2E16AE552E16EC2
:100CF000E552E7CFD9FF120001010251070A01E1D5
:100D00007DD0010A6CE0030A58E0010A47E0070AB7
:100D10003EE0010A21E0030A0AE0010A01E07FD077
:100D20000101CD519212CE519312CF5144D00351B3
:100D30000101CD15926E010104510101CE15936E92
:100D4000010105510101CF15946E010106A102D0E8
:100D5000F19E65D0F18E63D003510101CD15106E67
:100D6000CD1D89141010896E010104510101CE15A9
:100D7000106ECE1D8A1410108A6E010105510101FA
:100D8000CF15106ECF1D8B1410108B6E48D080CFF6
:100D900003F181CF04F182CF05F141D0035101016C
:100DA000CD159212010104510101CE1593120101DA
:100DB00005510101CF15941232D003510101CD1517
:100DC000E81C9216010104510101CE15E81C93168E
:100DD000010105510101CF15E81C941620D00351E3
:100DE0000101CD158912010104510101CE158A12AC
:100DF000010105510101CF158B1211D003510101E1
:100E0000CD15E81C8916010104510101CE15E81C1D
:100E10008A16010105510101CF15E81C8B1601014D
:100E2000100E006F1200D9CFE6FFE1CFD9FFE652D6
:100E300001010251030A01E1DFD0010A01E1C8D03A
:100E4000030A0EE0010A01E0DED0C26A0F0EC16E95
:100E50000101D051CD13D151CE13D06BD16BD3D072
:100E6000C26AAA0EC06E03510A0A01E191D0030AB8
:100E700001E17ED0010A6CE00F0A5AE0010A49E064
:100E8000030A3EE0010A32E0070A26E0010A1AE0FE
:100E9000030A0FE0010A01E08AD00F0EC16ED00EE6
:100EA0000101CD152F09CD6FE00ECE151F09CE6FB4
:100EB0007ED092800101D081D00ECD152E09CD6F4C
:100EC0000E0E74D0030E92120101D013D00ECD1568
:100ED0002C09CD6F0D0E6AD0070E92120101D013AE
:100EE000D00ECD152809CD6F0C0E60D00F0E9212CA
:100EF0000101D013D00ECD152009CD6F0B0E56D0A9
:100F00002F0E92120101D013D00ECD15CD6F0A0E07
:100F10004DD02F0E92120101D013D00ECD15CD6FF2
:100F20009384D185E00ECE151B09CE6F060E3ED000
:100F30002F0E92120101D013D00ECD15CD6F0C0ED5
:100F40009312D113E00ECE151309CE6F050E2ED0DD
:100F50002F0E92120101D013D00ECD15CD6F0E0EB3
:100F60009312D113E00ECE151109CE6F040E1ED0D0
:100F70002F0E92120101D013D00ECD15CD6F1E0E83
:100F80009312D113E00ECE150109CE6F030E0ED0D1
:100F90002F0E92120101D013D00ECD15CD6F1F0E62
:100FA0009312D113E00ECE15CE6F020EC16E010169
:100FB0000451030A08E0010A04E0030A06E1C188BB
:100FC00004D0C18A02D0300EC112010EC26E1BD0F5
:100FD00003C1DFFFDF50040802E2030EDF26DF500B
:100FE000040DF3500109C26E280EE66EE66ADAECD3
:100FF00021F0E552E55207D0C282C2B2FED7C3CF7C
:1010000003F1C4CF04F10101100E006FE552E55267
:10101000E7CFD9FF1200D9CFE6FFE1CFD9FF0B0E02
:10102000E12601010251050A63E0060A07E0010A10
:1010300001E1AAD1030A01E1A7D1A6D19288035107
:10104000080A20E00F0A1CE0010A18E0030A14E075
:10105000010A10E0070A0CE0010A08E0030A04E0B4
:10106000010A12E1200E0FD0210E0DD0220E0BD05E
:10107000230E09D0240E07D0250E05D0260E03D04E
:10108000270E01D0280ED56ED76AD66AF294D58E77
:101090000451030A10E0010A08E0030A04E0010A0F
:1010A0001FE10A0E03D0010E01D00A0EE66EE66AB9
:1010B00036EC22F013D0630EE66EE66A36EC22F0D0
:1010C000E552E552E668030EE66EDAEC21F0E552F1
:1010D000E5520C0EE66EE66ADAEC21F0E552E552D6
:1010E000D59ED6CF03F1D7CF04F1F2A44DD14AD18A
:1010F0009288270ED56ED76AD66AF294D58E010EE5
:10110000E66EE66A36EC22F0E552E552D59E080E10
:10111000D6CFDBFFDB50106E116A113408E210509D
:101120009C08000E115403E2260ED56E48D0080E1E
:10113000DB50106E116A113409E210509C08000E49
:10114000115404E2260ED56E800E33D0080EDB500B
:101150004E0804E2250ED56E400E2BD0080EDB5053
:10116000270804E2240ED56E200E23D0080EDB5093
:10117000130804E2230ED56E100E1BD0080EDB50B0
:10118000090804E2220ED56E080E13D0080EDB50BB
:10119000040804E2210ED56E040E0BD0080EDB50BD
:1011A000020804E2200ED56E020E03D0280ED56E82
:1011B000010EF36E090EF3CFDBFF0A0EDB6AD76A6E
:1011C000D66AF294D58E630EE66EE66A36EC22F0AD
:1011D000E552E552E668030EE66EDAEC21F0E552E0
:1011E000E5520C0EE66EE66ADAEC21F0E552E552C5
:1011F000D59E040ED6CFDBFF050EDB6A060EDB6A3A
:10120000070EDB6A000ED7CFDFFF010EDB6A020E8E
:10121000DB6A030EDB6AD9CFE9FFDACFEAFFEF50D2
:10122000EE6AEFCFF4FFEE6EEF50F4CFEEFFEF6E0D
:10123000D9CFE9FFDACFEAFF040EDB50EE26050E28
:10124000DB50EE22060EDB50EE22070EDB50EE22C4
:10125000D9CFE9FFDACFEAFF0A0E096E0A6A0B6AF4
:101260000C6AEECF04F0EECF05F0EECF06F0EFCF34
:1012700007F0C7EC28F003C0EDFF02C0EDFF01C08E
:10128000EDFF00C0EFFF090EDBCF10F00A0EDBCF41
:1012900011F0126A136AD9CFE9FFDACFEAFF10C062
:1012A00009F011C00AF012C00BF013C00CF0EECF21
:1012B00004F0EECF05F0EECF06F0EFCF07F0C7EC6D
:1012C00028F003C0EDFF02C0EDFF01C0EDFF00C03C
:1012D000EFFFD9CFE9FFDACFEAFFEECF10F01050E1
:1012E0000101036F106A1168126A136AD9CFE9FF0E
:1012F000DACFEAFFEE501016EE501116EE5012162D
:10130000EE501316080ED8901332123211321032EA
:10131000E806F9E110C004F1106A116A1268136A54
:10132000D9CFE9FFDACFEAFFEE501016EE501116D2
:10133000EE501216EE501316100ED89013321232D1
:1013400011321032E806F9E110C005F1106A116A95
:10135000126A1368D9CFE9FFDACFEAFFEE50101610
:10136000EE501116EE501216EE501316180ED890BD
:101370001332123211321032E806F9E110C006F1D0
:10138000F2A402D0010101690101100E006F0B0EE1
:10139000E15C02E2E16AE552E16EE552E7CFD9FF96
:1013A0001200D9CFE6FFE1CFD9FF030EE1263C0EB4
:1013B000DF6E01010251070A01E109D1010A01E1D1
:1013C00003D1030A01E19CD0010A01E17AD0070AA6
:1013D0004CE0010A42E0030A0DE0010A01E0F9D005
:1013E0004F0EAB16AC9ACF0E9D16C00E0101CF1357
:1013F000D76BEFD00F0E0315040A14E0070A0CE0B8
:10140000010A08E0030A04E0010A17E19B0E05D077
:10141000190E03D0330E01D09B0EE66EE66ADFCFC5
:10142000E6FF06D04D0EE66EE66AEF0EDF14E66EBE
:101430000EEC28F0E552E552E552010103BF03D05E
:10144000CF0EB81402D0300EB810B86E3F0E0101A6
:10145000CF17D86B010ED76FBCD0ACA2FED703C19B
:10146000E6FF13EC2BF0E552B4D00101D85126E091
:10147000AAC103F1010EDB6AD851F36E010EDBCF76
:10148000F4FFF350F45C16E2010EDB28EA6AAA0FBF
:10149000E96E010EEA22EF50E66E010EDB50EA6AB9
:1014A000AA0FE96E010EEA22E552E750EF6E010E37
:1014B000DB2AE2D7D8070101016B8BD0010101695A
:1014C00088D0DE52030EDD6E030E01010325F36E9C
:1014D000010EDBCFF4FFF350F45C01E37AD0ACA251
:1014E000FED7010EDB50EA6A010FE96E010EEA2217
:1014F000EF50E66E13EC2BF0E552010EDB2AE4D739
:101500000101D8515EE0020E03C1DBFFDB500D0884
:1015100005E20D0EF36E020EF3CFDBFF020EDBCF02
:1015200010F0D851D880105403E2020ED8C1DBFF6E
:10153000010EDB6AD851F36E010EDBCFF4FFF350DE
:10154000F45C38E2020EDB50F36E010EDBCFF4FFE9
:10155000F350F45C14E2010EDB50EA6AAA0FE96E64
:10156000010EEA22EF50E66E010EDB50030FEA6A2D
:10157000010FE96E010EEA22E552E750EF6E020E0E
:10158000DBCFE6FF010EDB50E552E724EA6AAA0F43
:10159000E96E010EEA22EF50E66E010EDB50EA6AB8
:1015A000AA0FE96E010EEA22E552E750EF6E010E36
:1015B000DB2AC0D7020EDB50D85F020EDBCF03F16F
:1015C00008D00101036B05D0D8C103F102D001019D
:1015D000D86B0101100E006F030EE15C02E2E16ABC
:1015E000E552E16EE552E7CFD9FF12000101D85173
:1015F000106E116A200E105C000E115801E31200EB
:101600009EAA0ED0B0EC29F0E66E0101D851D82B7D
:10161000EA6AAA0FE96E010EEA22E552E750EF6E80
:1016200000016AA702D0AB98AB881200D9CFE6FFC1
:10163000E1CFD9FFE652DF6A0A0EDF5C02E3000E5B
:1016400001D0010E106E9E50080B080A01E0010E39
:10165000101409E0640EE66EE66ADAEC21F0E55259
:10166000E552DF2AE9D70A0EDF5C02E3FF0E02D063
:101670009E96000EE552E552E7CFD9FF12009E96E6
:10168000C58016EF0BF0C5841200D9CFE6FFE1CF7D
:10169000D9FFFE0EDBCFE6FF8EEC28F0E55287EC9B
:1016A0002BF0E552E7CFD9FF1200D9CFE6FFE1CF0B
:1016B000D9FFFD0EDBCFF3FFDB06F35000091FE07F
:1016C0006FEC2BF0E66EFE0EDB50EA6A010FE96E5E
:1016D000010EEA22E552E750EF6EFE0EDB2AC5B698
:1016E000FED7A1A602D0FF0E0BD0FD0EDB5002E00C
:1016F000C59A01D0C58AC588C5A8DBD7FDD7000E1D
:10170000E552E7CFD9FF1200D9CFE6FFE1CFD9FFED
:10171000FD0EDBCFF3FFDB06F350000930E0C6A679
:1017200017D0FE0EDB50EA6A010FE96E010EEA22C5
:10173000EF50E66E8EEC28F0E552000902E0FD0E57
:101740001FD0FE0EDB2A87EC2BF0C5ACE1D715D0FD
:101750009E96FE0EDB50EA6A010FE96E010EEA2248
:10176000EF50C96EFE0EDB2AC6889EA6FED7C75074
:10177000040BCEE1C750010BCBE1FE0E01D0000EF1
:10178000E552E7CFD9FF1200D9CFE6FFE1CFD9FF6D
:10179000020EE12601010251170A01E104D1010AFA
:1017A00001E1DFD0030A01E1CBD0010A01E1B4D0AD
:1017B000070A01E1A0D0010A01E18CD0150A6FE00F
:1017C000010A56E0030A48E0010A3BE0070A32E05A
:1017D000010A27E0030A08E0010A01E010D1C69AD5
:1017E000030E0101CE130BD13F0EC716C66AC56AA0
:1017F000C68693829380C68A770EC86E0451020A09
:1018000009E0030A05E0010A08E1C78E770E04D05B
:101810001D0E02D0C78E0B0EC86EFC0E0101CE1736
:10182000EED02DDF01010351E824E66E2EDFE552F4
:10183000010E81D024DF01010351E8240109E66E85
:1018400065D01DDF010E04C1DBFF01010351E82457
:10185000046F010EDB286FD012DF01010351E82471
:101860000109E66E12DFE55204C1E6FF040EC0D0A6
:1018700006DF01010351E824FE0BE66E06DFE552A8
:1018800005C1E6FF02DFE552FADE01010351E8245B
:101890000109E66EFADEE55204C1E6FF60D0EFDE34
:1018A00001010351E824FE0BE66EEFDEE55205C1AF
:1018B000E6FFEBDEE55206C1E6FFE7DEE552DFDEDE
:1018C00001010351E8240109E66EDFDEE55204C19F
:1018D000E6FF67D0D4DE030E01010315E824F0090A
:1018E000E66ED3DEE55204C1E6FFCFDEE552010E1F
:1018F000E66E040E22D0C3DE030E01010315E824B8
:10190000F109E66EC2DEE55204C1E6FFBEDEE55235
:10191000010EE66E020E6CD0B2DE010E05C1DBFFD9
:1019200004C105F1030E01010315E824F009046F59
:10193000010EDB50020FE66E030EE66EE5DE5AD0B6
:101940009EDE030E01010315E824F109E66E9DDE1B
:10195000E55204C1E6FF99DEE55205C1E6FF050E3A
:1019600047D08DDE030E01010315E824F009E66E71
:101970008CDEE55204C1E6FF88DEE55206C1E6FFD3
:1019800084DEE5527CDE030E01010315E824F10933
:10199000E66E7BDEE55204C1E6FF77DEE55205C167
:1019A000E6FF060E25D06BDE030E01010315E824C9
:1019B000F009E66E6ADEE55204C1E6FF66DEE55236
:1019C00006C1E6FF62DEE55207C1E6FF5EDEE552D4
:1019D00056DE030E01010315E824F109E66E55DE1B
:1019E000E55204C1E6FF51DEE55205C1E6FF070EF0
:1019F000E66E5BDEE552E5520101016F44DE010156
:101A0000100E006F020EE15C02E2E16AE552E16E47
:101A1000E552E7CFD9FF1200D9CFE6FFE1CFD9FFDA
:101A2000E652DF6AFE0EDB500F0B060A14E0030AD3
:101A300010E0010A0CE0070A08E0010A04E0030ACA
:101A40000CE1040E09D0080E07D0100E05D0200EB0
:101A500003D0400E01D0800EDF6EDF50E552E5521C
:101A6000E7CFD9FF1200D9CFE6FFE1CFD9FFFE0EB5
:101A7000DBCFE6FFD1DFE552E81C8A16E552E7CF5F
:101A8000D9FF1200D9CFE6FFE1CFD9FFFE0EDBCFA1
:101A9000E6FFC2DFE5528A12E552E7CFD9FF120016
:101AA000D9CFE6FFE1CFD9FF050EE12601010251B2
:101AB000040A01E1B9D0070A01E1ABD0010A01E152
:101AC00095D0030A0FE0010A01E0E5D0C69A030EA3
:101AD0000101CE13CF8FD25101E0CD8BD351CE1364
:101AE000D36BD9D00101D36B020EDF6E010EDB6A1E
:101AF000800EF36E020EF3CFDBFFD26B01010351B8
:101B0000060A19E0030A14E0010A0FE0070A0AE0D6
:101B1000010A05E0030A12E10101040E0ED00101E1
:101B20000C0E0BD001011C0E08D001013C0E05D09B
:101B300001017C0E02D00101FC0ED36F01010451A2
:101B4000060A14E0030A0CE0060A08E0010A04E0B1
:101B5000030A0EE1DF6A0CD0010E09D0020E07D095
:101B6000040EDF6E0101010ED26F02D0050EDF6E92
:101B700001010551040A0FE0070A0AE0010A05E025
:101B8000030A0CE1010EDB6A09D0DE52010E05D01A
:101B9000DE52020E02D0DE52030EDD6E0651020A44
:101BA00008E0030A08E1800EF36E020EF3CFDBFFBC
:101BB00002D0020EDB6A020EDBCFE6FF010EDBCFA6
:101BC000E6FFDFCFE6FFFFEC28F0E552E552E552F5
:101BD000FC0E0101CE17CF9FD25101E0CD9BD31D4A
:101BE000CE17D31D9316D3518A1255D003C1E6FFE9
:101BF0003ADFE5529E9604C1C9FFC6AE03D001018B
:101C0000046904D09EA6FED70101046B03BD43D036
:101C10003ED003C1E6FF27DFE5522AEC2BF001019D
:101C2000046F03BD38D033D0030E04C1DBFF046B57
:101C3000040EDB6E030EDB50040FF36E040EDBCFDD
:101C4000F4FFF350F45C20E203C1E6FF0CDFE55241
:101C50009E96040EDB50EA6A010FE96E010EEA223D
:101C6000EF50C96EC6AE03D00101046902D09EA632
:101C7000FED7800E0101035D04E303C1E6FF02DF2E
:101C8000E552040EDB2AD6D7010103BD04D003C1FF
:101C9000E6FFF8DEE5520101100E006F050EE15C73
:101CA00002E2E16AE552E16EE552E7CFD9FF1200A8
:101CB000D9CFE6FFE1CFD9FF020EE12601010251A3
:101CC000030A30E0010A23E0030A08E0010A39E1CF
:101CD000C69A030E0101CE13CF8F33D00351030AEE
:101CE0000CE0010A08E0030A04E0010A0BE1120E0D
:101CF00005D0100E03D0110E01D0120EE66ECCEC02
:101D00002AF0E552FC0E0101CE17CF9F1AD003C175
:101D1000E6FF9BEC2AF0E5520101040512E181B0D7
:101D200010D0FDD703C1DFFF010E04C1DBFFDBCF05
:101D3000E6FFDFCFE6FF0DEC2AF0E552E5520101A8
:101D4000036F0101100E006F020EE15C02E2E16A16
:101D5000E552E16EE552E7CFD9FF1200D9CFE6FF99
:101D6000E1CFD9FF040EE12601010251020A3FE052
:101D7000010A3DE0020A09E0010A01E0B2D0030EC7
:101D80000101CE13800ECF17ACD0030E0315010155
:101D9000D46F100E01010315E8380F0B0101D56F48
:101DA000C00E01010315C00A0FE0400A0AE0C00A94
:101DB00005E0400A0CE101010A0E08D00101640EA1
:101DC00005D00101E80E02D00101100ED66FFC0E05
:101DD0000101CE17CF9F93929380949ED40501E189
:101DE0007DD0030ED45D01E179D08A927AD0030EC2
:101DF000DF6E01010325DF5C6BE2DF50EA6A010F51
:101E0000E96E010EEA22020EEFCFDBFF030EDB6A62
:101E1000DE52800EDD6E010EDB5000084EE2010145
:101E2000D45103E0030ED45D02E18A8201D08A928C
:101E3000020EDBCFE6FF010EDB50E552E71402E0B5
:101E40008B8E01D08B9ED651E66EE66ADAEC21F0DD
:101E5000E552E5520101D5050BE18AA009D0030E38
:101E6000DBCFE7FF010EDB50E712030EE7CFDBFF0E
:101E7000D45103E0030ED45D02E18A9201D08A823C
:101E8000D651E66EE66ADAEC21F0E552E552010140
:101E9000D5510BE18AA009D0030EDBCFE7FF010E7D
:101EA000DB50E712030EE7CFDBFF010EDBCFF3FFC2
:101EB000F390F342F3CFDBFFAED7DF50EA6A010FB6
:101EC000E96E010EEA22030EDBCFEFFFDF2A91D786
:101ED0000101D40503E0030ED45D02E18A8201D042
:101EE0008A920101100E006F040EE15C02E2E16AC9
:101EF000E552E16EE552E7CFD9FF12000101015131
:101F0000560A04E0030A03E18A8001D08B80640E44
:101F1000E66EE66ADAEC21F0E552E55212000101C4
:101F20000151560A04E0030A03E18A9001D08B9024
:101F3000640EE66EE66ADAEC21F0E552E552120034
:101F4000D9CFE6FFE1CFD9FFE652F00E93128A8691
:101F50008A94640EE66EE66ADAEC21F0E552E55208
:101F6000CDDF8150DF6EDBDFC9DFD9DFDF8E010E11
:101F70000009F6E10F0E93168A96E552E552E7CF77
:101F8000D9FF1200D9CFE6FFE1CFD9FFFE0EDB501B
:101F9000F00B106E0F0E8A1410108A6EAFDFBFDFC9
:101FA000FE0EDB500F0B100DF3CF10F00F0E8A1446
:101FB000F3108A6EA3DFB3DFE552E7CFD9FF12003B
:101FC000D9CFE6FFE1CFD9FF8A84FE0EDBCFE6FF53
:101FD000D9DFE552E552E7CFD9FF1200D9CFE6FFAE
:101FE000E1CFD9FF8A94FE0EDBCFE6FFCBDFE552CF
:101FF000E552E7CFD9FF1200D9CFE6FFE1CFD9FFF5
:102000008A94FE0EDBCFE6FFBDDFE552E552E7CF57
:10201000D9FF1200D9CFE6FFE1CFD9FF020EE126AA
:1020200001010251060A01E100D1030A01E1EAD0EF
:10203000010A01E1D4D0070A01E1C2D0010A01E19D
:10204000BBD0030A14E0010A01E019D10151560A7C
:1020500007E0030A01E013D1FD0E9312010105D040
:102060009480FC0E93120101CF81CE1308D103C1DD
:10207000CAF104C1CBF10101CC6BCA0509E1100E14
:10208000CB5D06E10101020E036F0101010ECC6F71
:10209000140EE66EE66A36EC22F0E552E5523FDFBA
:1020A0008A988A9A8A9C8A9E8A948A96010101510A
:1020B000560A07E0030A0BE1020E93160101CE1740
:1020C00006D0030E931694900101CE17CE918A8804
:1020D0008A8A640EE66EE66ADAEC21F0E552E55291
:1020E0000DDF1DDF140EE66EE66A36EC22F0E552D7
:1020F000E55204DF14DF640EE66EE66ADAEC21F0E6
:10210000E552E552FBDE0BDF640EE66EE66ADAECC2
:1021100021F0E552E5528A988A8A640EE66EE66AF4
:10212000DAEC21F0E552E552E9DEF9DE0101035176
:10213000020A0CE0030A06E0010A0CE1280EE66E32
:102140005BDFE552200EE66E57DFE552280EE66EA5
:1021500053DFE552640EE66EE66ADAEC21F0E552F2
:10216000E552080EE66E48DFE552640EE66EE66A5A
:10217000DAEC21F0E552E552010EE66E3DDFE55264
:102180000A0EE66EE66A36EC22F0E552E552060EDD
:10219000E66E32DFE552640EE66EE66ADAEC21F0B6
:1021A000E552E5520C0EE66E27DFE552640EE66E50
:1021B000E66ADAEC21F011D003C1E6FF01DF5ED060
:1021C00003C1E6FF0BDFE552040E0101035D57E298
:1021D000030EE66EE66A36EC22F0E5524FD0030EAF
:1021E000DF6E030E01010325DF5C49E2DF50EA6A7E
:1021F000010FE96E010EEA22EF50E66EE1DEE552D4
:10220000DF2AEFD7030EDF6E030E01010325DF5C2B
:1022100036E2DF50EA6A010FE96E010EEA22EF5062
:10222000E66EDCDEE552DF2AEFD70351010804E257
:102230000101CB5101010427010E0315400DF3509C
:102240000425E76E010EE7CFDBFF0101CC5111E061
:10225000010E04C1DBFF0101045107080AE2380E38
:10226000106E010EDBCFE7FF1050E726010EE7CF1F
:10227000DBFF010EDB508009E66EB0DEE5520101A6
:10228000100E006F020EE15C02E2E16AE552E16EBF
:10229000E552E7CFD9FF1200D9CFE6FFE1CFD9FF52
:1022A000040EE12601010251020A5CE0030A08E083
:1022B000010A01E080D096EC2BF00101CF857BD0A4
:1022C000DE52400EDD6EFD0EDF6E0351090A30E076
:1022D000010A2AE00F0A24E0010A1EE0030A18E0BE
:1022E000010A12E0070A0DE0010A08E0030A03E010
:1022F000010A22E10DD0DE52180E08D0DE52180E6F
:1023000009D0DE52180E0AD0DE523F0EDD6E0AD022
:10231000DE523F0EDD6E0AD0DE523F0EDD6E0AD079
:10232000010EDB68FC0E07D0010EDB68FD0E03D04A
:10233000010EDB68FE0EDF6E010EE66EE66A60ECF3
:1023400029F0E552E5527F0EDF14E66E80EC2AF0AC
:10235000E552010EDBCFE6FFB4EC2AF0E5520101B5
:10236000CF9529D00451E66ED950020FE96EDACF2D
:10237000EAFFE552E750EE6EED6AD950020FE96EC2
:10238000DACFEAFFEE50ED6EEF6A0351106E116A7C
:10239000D950020FE96EDACFEAFF1050EE12115059
:1023A000ED12020EDBCFE6FF030EDBCFE6FF60ECA3
:1023B00029F0E552E5520101100E006F040EE15CB8
:1023C00002E2E16AE552E16EE552E7CFD9FF120081
:1023D000D9CFE6FFE1CFD9FF040EE126010102517A
:1023E000020A5CE0030A08E0010A01E080D094ECF4
:1023F0002BF00101CF837BD0DE52400EDD6EFD0E4F
:10240000DF6E0351090A30E0010A2AE00F0A24E0D6
:10241000010A1EE0030A18E0010A12E0070A0DE0B3
:10242000010A08E0030A03E0010A22E10DD0DE52AE
:10243000180E08D0DE52180E09D0DE52180E0AD03F
:10244000DE523F0EDD6E0AD0DE523F0EDD6E0AD048
:10245000DE523F0EDD6E0AD0010EDB68FC0E07D0A7
:10246000010EDB68FD0E03D0010EDB68FE0EDF6E91
:10247000010EE66EE66A31EC29F0E552E5527F0E78
:10248000DF14E66E80EC2AF0E552010EDBCFE6FFAA
:1024900053EC28F0E5520101CF9329D00451E66EA8
:1024A000D950020FE96EDACFEAFFE552E750EE6E3F
:1024B000ED6AD950020FE96EDACFEAFFEE50ED6E09
:1024C000EF6A0351106E116AD950020FE96EDACF2C
:1024D000EAFF1050EE121150ED12020EDBCFE6FFB4
:1024E000030EDBCFE6FF31EC29F0E552E5520101A6
:1024F000100E006F040EE15C02E2E16AE552E16E4B
:10250000E552E7CFD9FF1200D9CFE6FFE1CFD9FFDF
:10251000050EE12601010251050A71E0010A1DE0E4
:10252000070A13E0010A01E0B4D0A69EA69CA68487
:1025300003C1A9FF04C1A8FF550EA76EAA0EA76E7E
:10254000A682A1A8FED7A198A4D0A69EA69C03C14E
:10255000A9FFA680A8CF04F19CD0040EDF6E035122
:10256000E66ED950030FE96EDACFEAFFE552E75085
:10257000EE6EED6A0451106E116AD950030FE96EC8
:10258000DACFEAFF1050EE261150ED220351E66E2D
:10259000D950010FE96EDACFEAFFE552E750EE6E4F
:1025A000ED6A010EDBCF10F0020EDBCF11F0030E4F
:1025B000DBCF12F0040EDBCF13F01250105C13507F
:1025C000115867E2A69EA69CA684010EDB50A96E58
:1025D000DF50EA6A010FE96E010EEA22EF50A86EA1
:1025E000550EA76EAA0EA76EA682A1A8FED7A19827
:1025F000DF2A010EDB2A020ED4E3DB2AD2D7040E37
:10260000DF6E0351E66ED950030FE96EDACFEAFFB1
:10261000E552E750EE6EED6A0451106E116AD95022
:10262000030FE96EDACFEAFF1050EE261150ED22CB
:102630000351E66ED950010FE96EDACFEAFFE55299
:10264000E750EE6EED6A010EDBCF10F0020EDBCF2D
:1026500011F0030EDBCF12F0040EDBCF13F012509B
:10266000105C1350115815E2A69EA69C010EDB507B
:10267000A96EA680DF50EA6A010FE96E010EEA2218
:10268000A8CFEFFFDF2A010EDB2A020EDCE3DB2AF4
:10269000DAD70101100E006F050EE15C02E2E16A7B
:1026A000E552E16EE552E7CFD9FF1200D9CFE6FF40
:1026B000E1CFD9FFE652FE0EDB50100DF3CFE9FF5C
:1026C000F4CFEAFF410EE926010EEA22EFCFDFFF49
:1026D000FE0EDB50100DF3CFE9FFF4CFEAFF410E01
:1026E000E926010EEA22020EE926000EEA22EF5048
:1026F000800B02E0000EDF80070EDF14070A1CE0EB
:10270000010A18E0030A14E0010A10E0070A0CE0CD
:10271000010A08E0030A04E0010A0FE1350E0DD0BA
:10272000210E0BD0390E09D0180E07D03A0E05D065
:10273000220E03D0360E01D0140EE552E552E7CF3B
:10274000D9FF1200D9CFE6FFE1CFD9FFFE0EDB5053
:10275000100DF3CFE9FFF4CFEAFF410EE926010E99
:10276000EA22080EE926000EEA220A0EEF6EFE0E9D
:10277000DB50100DF3CFE9FFF4CFEAFF410EE9265D
:10278000010EEA22080EE926000EEA22010EE926D1
:10279000000EEA22080EEF6EFE0EDB50100DF3CF96
:1027A000E9FFF4CFEAFF410EE926010EEA22080E06
:1027B000E926000EEA22020EE926000EEA22070EA2
:1027C000EF6EFE0EDB50100DF3CFE9FFF4CFEAFF02
:1027D000410EE926010EEA22080EE926000EEA2241
:1027E000030EE926000EEA22060EEF6EFE0EDB5007
:1027F000100DF3CFE9FFF4CFEAFF410EE926010EF9
:10280000EA22080EE926000EEA22040EE926000E4E
:10281000EA22050EEF6EFE0EDB50100DF3CFE9FF3E
:10282000F4CFEAFF410EE926010EEA22080EE9265E
:10283000000EEA22050EE926000EEA22040EEF6ED3
:10284000FE0EDB50100DF3CFE9FFF4CFEAFF410E8F
:10285000E926010EEA22080EE926000EEA22060EFB
:10286000E926000EEA22030EEF6EFE0EDB50100D7D
:10287000F3CFE9FFF4CFEAFF410EE926010EEA2289
:10288000080EE926000EEA22070EE926000EEA22CB
:10289000020EEF6EE552E7CFD9FF1200D9CFE6FF67
:1028A000E1CFD9FFFD0EDB50040A20E0070A15E056
:1028B000010A08E0030A29E1FE0EDB500F0B106E3F
:1028C000F00E07D0FE0EDB500F0B100DF3CF10F003
:1028D0000F0E8A141010816E18D0FE0EDB500F0BF5
:1028E000106EF00E89141010806E0FD0FE0EDB50AB
:1028F000080DF350400B116EFE0EDB50070B106EEF
:10290000B80E8B1410101110826EE552E7CFD9FF6C
:102910001200D9CFE6FFE1CFD9FF040EE126020E67
:10292000DB6A030EDB6AFE0EDB50100DF3CFE9FF0E
:10293000F4CFEAFF410EE926010EEA22030EE92652
:10294000000EEA22EF50DE6EDD6AFE0EDB50100D47
:10295000F3CFE9FFF4CFEAFF410EE926010EEA22A8
:10296000020EE926000EEA22EF50200B01E1B5D05D
:10297000FE0EDB50100DF3CFE9FFF4CFEAFF410E5E
:10298000E926010EEA22060EE926000EEA22EECF23
:1029900010F0EFCF11F0D890115004E6080E105C43
:1029A000000E11582DE2FE0EDB50100DF3CFE9FFA3
:1029B000F4CFEAFF410EE926010EEA22080EE926CD
:1029C000000EEA22E9CF10F0EACF11F0FE0EDB5044
:1029D000100DF3CFE9FFF4CFEAFF410EE926010E17
:1029E000EA22060EE926000EEA221050EE24E76ED7
:1029F0001150EE20EA6EE7CFE9FF020EEFCFDBFFCA
:102A0000FE0EDB50100DF3CFE9FFF4CFEAFF410ECD
:102A1000E926010EEA22040EE926000EEA22EECF94
:102A200010F0EFCF11F0D890115004E6080E105CB2
:102A3000000E11582DE2FE0EDB50100DF3CFE9FF12
:102A4000F4CFEAFF410EE926010EEA22080EE9263C
:102A5000000EEA22E9CF10F0EACF11F0FE0EDB50B3
:102A6000100DF3CFE9FFF4CFEAFF410EE926010E86
:102A7000EA22040EE926000EEA221050EE24E76E48
:102A80001150EE20EA6EE7CFE9FF030EEFCFDBFF38
:102A9000DECF10F0DDCF11F0020EDB50000111AEE1
:102AA00002D0D89003D0105C000E115804E2020E40
:102AB000DB50DE6EDD6ADECF10F0DDCF11F0030EED
:102AC000DB5011AE02D0D89003D0105C000E11582C
:102AD00004E2030EDB50DE6EDD6AFE0EDB50100DED
:102AE000F3CFE9FFF4CFEAFF410EE926010EEA2217
:102AF000060EE926000EEA22EE2AEF22FE0EDB5039
:102B0000100DF3CFE9FFF4CFEAFF410EE926010EE5
:102B1000EA22020EE926000EEA22EF50400B14E0F2
:102B2000DECF10F0DDCF11F0640E1102F3CF11F003
:102B30001002F3CF10F0F4501126F3CFE6FF11C0CE
:102B4000E6FFDAEC21F006D0DECFE6FFDDCFE6FFD0
:102B500036EC22F0E552E552040EE15C02E2E16A55
:102B6000E552E16EE552E7CFD9FF1200D9CFE6FF7B
:102B7000E1CFD9FF01010251040A01E198D2070A0D
:102B800001E15BD2010A5CE0030A24E0010A02E0F1
:102B9000FFEF19F0FE0EDB50040A16E0070A0EE004
:102BA000010A06E0030A02E0FFEF19F00F0E01D060
:102BB000F00E93120101CE13FFEF19F00F0E9212D7
:102BC0000101CD13FFEF19F0470E94120101CF134D
:102BD000FFEF19F0FE0EDBCFE6FFDBCFE9FFEA6A7D
:102BE000E9BEEA68040ED890E936EA36E806FBE169
:102BF000410EE926010EEA22EF50E66E57DDE5525E
:102C0000E66E4CDEE552E552FE0EDB50040A13E0A0
:102C1000070A0CE0010A05E0030A01E0F0D3F00E18
:102C200001D00F0E93160101CE17E9D3F00E9216C4
:102C30000101CD17E4D3B80E94160101CF17DFD3ED
:102C4000065102E1010E066FFE0EDBCFE9FFEA6AD4
:102C5000E9BEEA68040ED890E936EA36E806FBE1F8
:102C6000410EE926010EEA22EE52010EEF6EFE0E33
:102C7000DBCFE9FFEA6AE9BEEA68040ED890E936DC
:102C8000EA36E806FBE1410EE926010EEA22020ED1
:102C9000E926000EEA2205C1EFFFFE0EDBCFE9FFB9
:102CA000EA6AE9BEEA68040ED890E936EA36E80630
:102CB000FBE1410EE926010EEA22030EE926000E91
:102CC000EA2206C1EFFF01010451E66EFE0EDBCFE2
:102CD000E9FFEA6AE9BEEA68040ED890E936EA3606
:102CE000E806FBE1410EE926010EEA22040EE92680
:102CF000000EEA22E552E750EE6EED6AFE0EDBCFE3
:102D0000E9FFEA6AE9BEEA68040ED890E936EA36D5
:102D1000E806FBE1410EE926010EEA22040EE9264F
:102D2000000EEA22EE50ED6EEF6A01010351106EC3
:102D3000116AFE0EDBCFE9FFEA6AE9BEEA68040E1B
:102D4000D890E936EA36E806FBE1410EE926010EA5
:102D5000EA22040EE926000EEA221050EE26115057
:102D6000ED22FE0EDBCFE9FFEA6AE9BEEA68040E57
:102D7000D890E936EA36E806FBE1410EE926010E75
:102D8000EA22060EE926000EEA22EE6AED6AFE0E3F
:102D9000DBCFE9FFEA6AE9BEEA68040ED890E936BB
:102DA000EA36E806FBE1410EE926010EEA22020EB0
:102DB000E926000EEA22EF50020B020811E1FE0E96
:102DC000DBCFE9FFEA6AE9BEEA68040ED890E9368B
:102DD000EA36E806FBE1410EE926010EEA22EF9011
:102DE000FE0EDBCFE9FFEA6AE9BEEA68040ED8907E
:102DF000E936EA36E806FBE1410EE926010EEA2251
:102E0000020EE926000EEA22EF50040B040801E04E
:102E1000F6D2FE0EDBCFE9FFEA6AE9BEEA68040EED
:102E2000D890E936EA36E806FBE1410EE926010EC4
:102E3000EA22040EE926000EEA22EECF10F0EFCFD0
:102E400011F0113401E3ABD010500008000E115402
:102E500001E3A5D0FE0EDBCFE9FFEA6AE9BEEA682E
:102E6000040ED890E936EA36E806FBE1410EE92681
:102E7000010EEA22020EE926000EEA22EF50030BB1
:102E8000030A43E0010A1EE0030A0FE0010A5FE1C2
:102E9000FE0EDBCFE9FFEA6AE9BEEA68040ED890CD
:102EA000E936EA36E806FBE12AD0FE0EDBCFE9FF81
:102EB000EA6AE9BEEA68040ED890E936EA36E8061E
:102EC000FBE140D0FE0EDBCFE9FFEA6AE9BEEA682B
:102ED000040ED890E936EA36E806FBE1410EE92611
:102EE000010EEA22EF2AFE0EDBCFE9FFEA6AE9BE15
:102EF000EA68040ED890E936EA36E806FBE1410EAE
:102F0000E926010EEA22EF2A22D0FE0EDBCFE9FFEE
:102F1000EA6AE9BEEA68040ED890E936EA36E806BD
:102F2000FBE1410EE926010EEA22EF06FE0EDBCFA1
:102F3000E9FFEA6AE9BEEA68040ED890E936EA36A3
:102F4000E806FBE1410EE926010EEA22EF06FE0E3D
:102F5000DBCFE6FFDBCFE6FF56EC13F0E552E66E83
:102F60009DDCE552E552FE0EDBCFE6FFD2DCE552FA
:102F7000FE0EDBCFE9FFEA6AE9BEEA68040ED890EC
:102F8000E936EA36E806FBE1410EE926010EEA22BF
:102F9000040EE926000EEA22EE06EF5A3AD7FE0E9C
:102FA000DBCFE9FFEA6AE9BEEA68040ED890E936A9
:102FB000EA36E806FBE1410EE926010EEA22EE526E
:102FC000EF6AFE0EDBCFE9FFEA6AE9BEEA68040EAB
:102FD000D890E936EA36E806FBE1410EE926010E13
:102FE000EA22020EE926000EEA22EF50080B08083A
:102FF00001E005D2FE0EDBCFE9FFEA6AE9BEEA682E
:10300000040ED890E936EA36E806FBE1410EE926DF
:10301000010EEA22030EE926000EEA22EF500A0F03
:10302000E66EE66A36EC22F0E552E552FE0EDBCFA4
:10303000E6FFE66A33DCE55248D0FE0EDBCFE9FF5F
:10304000EA6AE9BEEA68040ED890E936EA36E8068C
:10305000FBE1410EE926010EEA22040EE926000EEC
:10306000EA22EECF10F010500101036FFE0EDBCF0D
:10307000E9FFEA6AE9BEEA68040ED890E936EA3662
:10308000E806FBE1410EE926010EEA22040EE926DC
:10309000000EEA22EECF10F0EFCF11F01016FF0E67
:1030A000111611C010F0116A10C004F1A8D103511B
:1030B000030A01E1D8D0010A0AE0020A01E09FD127
:1030C000FE0EDBCFE6FFA2EC13F0E55298D1FE0E28
:1030D000DBCFE9FFEA6AE9BEEA68040ED890E93678
:1030E000EA36E806FBE1410EE926010EEA22080E67
:1030F000E926000EEA2204C1EFFFFE0EDBCFE9FF56
:10310000EA6AE9BEEA68040ED890E936EA36E806CB
:10311000FBE1410EE926010EEA22080EE926000E27
:10312000EA22010EE926000EEA2205C1EFFFFE0E9B
:10313000DBCFE9FFEA6AE9BEEA68040ED890E93617
:10314000EA36E806FBE1410EE926010EEA22080E06
:10315000E926000EEA22020EE926000EEA2206C146
:10316000EFFFFE0EDBCFE9FFEA6AE9BEEA68040E74
:10317000D890E936EA36E806FBE1410EE926010E71
:10318000EA22080EE926000EEA22030EE926000EC6
:10319000EA2207C1EFFFFE0EDBCFE9FFEA6AE9BED4
:1031A000EA68040ED890E936EA36E806FBE1410EFB
:1031B000E926010EEA22080EE926000EEA22040E94
:1031C000E926000EEA2208C1EFFFFE0EDBCFE9FF81
:1031D000EA6AE9BEEA68040ED890E936EA36E806FB
:1031E000FBE1410EE926010EEA22080EE926000E57
:1031F000EA22050EE926000EEA2209C1EFFFFE0EC3
:10320000DBCFE9FFEA6AE9BEEA68040ED890E93646
:10321000EA36E806FBE1410EE926010EEA22080E35
:10322000E926000EEA22060EE926000EEA220AC16D
:10323000EFFFFE0EDBCFE9FFEA6AE9BEEA68040EA3
:10324000D890E936EA36E806FBE1410EE926010EA0
:10325000EA22080EE926000EEA22070EE926000EF1
:10326000EA220BC1EFFFFE0EDBCFE9FFEA6AE9BEFF
:10327000EA68040ED890E936EA36E806FBE1410E2A
:10328000E926010EEA22080EE926000EEA22EFCF17
:1032900004F1FE0EDBCFE9FFEA6AE9BEEA68040E3C
:1032A000D890E936EA36E806FBE1410EE926010E40
:1032B000EA22080EE926000EEA22010EE926000E97
:1032C000EA22EFCF05F1FE0EDBCFE9FFEA6AE9BEA5
:1032D000EA68040ED890E936EA36E806FBE1410ECA
:1032E000E926010EEA22080EE926000EEA22020E65
:1032F000E926000EEA22EFCF06F1FE0EDBCFE9FF52
:10330000EA6AE9BEEA68040ED890E936EA36E806C9
:10331000FBE1410EE926010EEA22080EE926000E25
:10332000EA22030EE926000EEA22EFCF07F1FE0E95
:10333000DBCFE9FFEA6AE9BEEA68040ED890E93615
:10334000EA36E806FBE1410EE926010EEA22080E04
:10335000E926000EEA22040EE926000EEA22EFCF4B
:1033600008F1FE0EDBCFE9FFEA6AE9BEEA68040E67
:10337000D890E936EA36E806FBE1410EE926010E6F
:10338000EA22080EE926000EEA22050EE926000EC2
:10339000EA22EFCF09F1FE0EDBCFE9FFEA6AE9BED0
:1033A000EA68040ED890E936EA36E806FBE1410EF9
:1033B000E926010EEA22080EE926000EEA22060E90
:1033C000E926000EEA22EFCF0AF1FE0EDBCFE9FF7D
:1033D000EA6AE9BEEA68040ED890E936EA36E806F9
:1033E000FBE1410EE926010EEA22080EE926000E55
:1033F000EA22070EE926000EEA22EFCF0BF10101C7
:10340000100E006FE552E7CFD9FF1200D9CFE6FFCB
:10341000E1CFD9FFFE0EDBCFE9FFEA6AE9BEEA6839
:10342000040ED890E936EA36E806FBE1410EE926BB
:10343000010EEA22040EE926000EEA22EECF10F079
:10344000EFCF11F0113401E3ACD010500008000EA2
:10345000115401E3A6D0FE0EDBCFE9FFEA6AE9BE14
:10346000EA68040ED890E936EA36E806FBE1410E38
:10347000E926010EEA22020EE926000EEA22EF50AA
:10348000030B030A43E0010A1EE0030A0FE0010AEE
:103490005FE1FE0EDBCFE9FFEA6AE9BEEA68040EEF
:1034A000D890E936EA36E806FBE12AD0FE0EDBCFFB
:1034B000E9FFEA6AE9BEEA68040ED890E936EA361E
:1034C000E806FBE140D0FE0EDBCFE9FFEA6AE9BE89
:1034D000EA68040ED890E936EA36E806FBE1410EC8
:1034E000E926010EEA22EF2AFE0EDBCFE9FFEA6AA7
:1034F000E9BEEA68040ED890E936EA36E806FBE150
:10350000410EE926010EEA22EF2A22D0FE0EDBCF81
:10351000E9FFEA6AE9BEEA68040ED890E936EA36BD
:10352000E806FBE1410EE926010EEA22EF06FE0E57
:10353000DBCFE9FFEA6AE9BEEA68040ED890E93613
:10354000EA36E806FBE1410EE926010EEA22EF0623
:10355000FE0EDBCFE6FFDBCFE6FF56EC13F0E552C5
:10356000E66E4EEC14F0E552E552FE0EDBCFE6FFC0
:1035700089EC14F0E552FE0EDBCFE9FFEA6AE9BE02
:10358000EA68040ED890E936EA36E806FBE1410E17
:10359000E926010EEA22040EE926000EEA22EE06D2
:1035A000EF5AFE0EDBCFE9FFEA6AE9BEEA68040ED5
:1035B000D890E936EA36E806FBE1410EE926010E2D
:1035C000EA22040EE926000EEA22EECF10F0EFCF39
:1035D00011F0113404E210500008000E11544EE3B3
:1035E000FE0EDBCFE9FFEA6AE9BEEA68040ED89076
:1035F000E936EA36E806FBE1410EE926010EEA2249
:10360000EE52EF6AFE0EDBCFE9FFEA6AE9BEEA6836
:10361000040ED890E936EA36E806FBE1410EE926C9
:10362000010EEA22020EE926000EEA22EF50080BF4
:10363000080824E1FE0EDBCFE9FFEA6AE9BEEA688A
:10364000040ED890E936EA36E806FBE1410EE92699
:10365000010EEA22030EE926000EEA22EF500A0FBD
:10366000E66EE66A36EC22F0E552E552FE0EDBCF5E
:10367000E6FFE66A4EEC14F0E552E552E552E7CF7C
:10368000D9FF1200D9CFE6FFE1CFD9FF020EE12624
:1036900001010251030A01E1FED1010A31E0030AEE
:1036A00019E0010A01E035D2FE0EDB50040A0DE0FC
:1036B000070A09E0010A05E0030A01E02AD2030E25
:1036C00005D00C0E03D0300E01D0C00E93120101B4
:1036D000CE131FD2FE0EDB50040A0DE0070A09E0EC
:1036E000010A05E0030A01E014D2FC0E05D0F30E36
:1036F00003D0CF0E01D03F0E93160101CE1709D291
:10370000065102E1010E066FFE0EDBCFE9FFEA6A09
:10371000E9BEEA68050EEA02F3CFEAFFE902F3CF59
:10372000E9FFF450EA26910EE926010EEA22010E85
:10373000EF6EFE0EDBCFE9FFEA6AE9BEEA68050E2E
:10374000EA02F3CFEAFFE902F3CFE9FFF450EA26F9
:10375000910EE926010EEA22EE5205C1EFFFFE0EA0
:10376000DBCFE9FFEA6AE9BEEA68050EEA02F3CFB9
:10377000EAFFE902F3CFE9FFF450EA26910EE926C9
:10378000010EEA22020EE926000EEA2206C1EFFF30
:103790000451E66EFE0EDBCFE9FFEA6AE9BEEA6895
:1037A000050EEA02F3CFEAFFE902F3CFE9FFF45096
:1037B000EA26910EE926010EEA22030EE926000E02
:1037C000EA22E552E750EE6EED6AFE0EDBCFE9FF2E
:1037D000EA6AE9BEEA68050EEA02F3CFEAFFE90207
:1037E000F3CFE9FFF450EA26910EE926010EEA2212
:1037F000030EE926000EEA22EE50ED6EEF6A035149
:10380000106E116AFE0EDBCFE9FFEA6AE9BEEA68D4
:10381000050EEA02F3CFEAFFE902F3CFE9FFF45025
:10382000EA26910EE926010EEA22030EE926000E91
:10383000EA221050EE261150ED22FE0EDB50040A53
:1038400057E0070A3AE0010A1DE0030A6BE1FE0EA9
:10385000DBCFE9FFEA6AE9BEEA68050EEA02F3CFC8
:10386000EAFFE902F3CFE9FFF450EA26910EE926D8
:10387000010EEA22EE52EF50010B02E08A8252D092
:103880008A9250D0FE0EDBCFE9FFEA6AE9BEEA6811
:10389000050EEA02F3CFEAFFE902F3CFE9FFF450A5
:1038A000EA26910EE926010EEA22EE52EF50010BB4
:1038B00002E08A8637D08A9635D0FE0EDBCFE9FF4C
:1038C000EA6AE9BEEA68050EEA02F3CFEAFFE90216
:1038D000F3CFE9FFF450EA26910EE926010EEA2221
:1038E000EE52EF50010B02E08A8A1CD08A9A1AD05D
:1038F000FE0EDBCFE9FFEA6AE9BEEA68050EEA02DE
:10390000F3CFEAFFE902F3CFE9FFF450EA26910E84
:10391000E926010EEA22EE52EF50010B02E08A8EF8
:1039200001D08A9EFE0EDBCFE9FFEA6AE9BEEA68B3
:10393000050EEA02F3CFEAFFE902F3CFE9FFF45004
:10394000EA26910EE926010EEA22EE52EF50040B10
:10395000040801E0DED0FE0EDBCFE9FFEA6AE9BE33
:10396000EA68050EEA02F3CFEAFFE902F3CFE9FFC6
:10397000F450EA26910EE926010EEA22030EE9260A
:10398000000EEA22EECF10F0EFCF11F011346EE20C
:1039900010500008000E115469E2FE0EDB50040ABC
:1039A00024E0070A18E0010A0CE0030A27E18A90E4
:1039B000010EE66EE66ADAEC21F0E552E5528A8005
:1039C0001DD08A94010EE66EE66ADAEC21F0E5522B
:1039D000E5528A8413D08A98010EE66EE66ADAEC24
:1039E00021F0E552E5528A8809D08A9C010EE66EE4
:1039F000E66ADAEC21F0E552E5528A8CFE0EDBCF66
:103A0000E9FFEA6AE9BEEA68050EEA02F3CFEAFFD7
:103A1000E902F3CFE9FFF450EA26910EE926010E00
:103A2000EA22020EE926000EEA22EF50E66EE66A6E
:103A300036EC22F0E552E552FE0EDBCFE9FFEA6AF2
:103A4000E9BEEA68050EEA02F3CFEAFFE902F3CF26
:103A5000E9FFF450EA26910EE926010EEA22030E50
:103A6000E926000EEA22EE06EF5A75D7FE0EDBCFEE
:103A7000E9FFEA6AE9BEEA68050EEA02F3CFEAFF67
:103A8000E902F3CFE9FFF450EA26910EE926010E90
:103A9000EA22EF6A3ED0FE0EDBCFE9FFEA6AE9BE1A
:103AA000EA68050EEA02F3CFEAFFE902F3CFE9FF85
:103AB000F450EA26910EE926010EEA22030EE926C9
:103AC000000EEA22EECF10F01050036FFE0EDBCF97
:103AD000E9FFEA6AE9BEEA68050EEA02F3CFEAFF07
:103AE000E902F3CFE9FFF450EA26910EE926010E30
:103AF000EA22030EE926000EEA22EECF10F0EFCF05
:103B000011F01016FF0E111611C010F0116A10C03E
:103B100004F10101100E006F020EE15C02E2E16AA5
:103B2000E552E16EE552E7CFD9FF1200D9CFE6FFAB
:103B3000E1CFD9FFFE0EDBCFE9FFEA6AE9BEEA6812
:103B4000050EEA02F3CFEAFFE902F3CFE9FFF450F2
:103B5000EA26910EE926010EEA22030EE926000E5E
:103B6000EA22EECF10F0EFCF11F011346DE21050D9
:103B70000008000E115468E2FE0EDB50040A24E037
:103B8000070A18E0010A0CE0030A27E18A90010EF7
:103B9000E66EE66ADAEC21F0E552E5528A801DD045
:103BA0008A94010EE66EE66ADAEC21F0E552E552FF
:103BB0008A8413D08A98010EE66EE66ADAEC21F068
:103BC000E552E5528A8809D08A9C010EE66EE66AC3
:103BD000DAEC21F0E552E5528A8CFE0EDBCFE9FFEC
:103BE000EA6AE9BEEA68050EEA02F3CFEAFFE902F3
:103BF000F3CFE9FFF450EA26910EE926010EEA22FE
:103C0000020EE926000EEA22EF50E66EE66A36EC76
:103C100022F0E552E552FE0EDBCFE9FFEA6AE9BE8B
:103C2000EA68050EEA02F3CFEAFFE902F3CFE9FF03
:103C3000F450EA26910EE926010EEA22030EE92647
:103C4000000EEA22EE06EF5AFE0EDBCFE9FFEA6A2B
:103C5000E9BEEA68050EEA02F3CFEAFFE902F3CF14
:103C6000E9FFF450EA26910EE926010EEA22030E3E
:103C7000E926000EEA22EECF10F0EFCF11F011345A
:103C800004E210500008000E115414E3FE0EDBCFC6
:103C9000E9FFEA6AE9BEEA68050EEA02F3CFEAFF45
:103CA000E902F3CFE9FFF450EA26910EE926010E6E
:103CB000EA22EF6AE552E7CFD9FF12000101025173
:103CC000030A2EE0010A1BE0030A0FE0010A2EE1BD
:103CD0000101DA6BD96B320EDB6FDC6FDD6FDE6FEB
:103CE000DF6FE06FE16FE26F21D003C1DAF1010114
:103CF000DA5102E1000E01D0010ED96F17D003C1D5
:103D0000DBF104C1DCF105C1DDF106C1DEF107C163
:103D1000DFF108C1E0F109C1E1F10AC1E2F106D029
:103D20000351050DF3CFEDF1F4CFEEF10101100ECB
:103D3000006F120001010251030A2EE0010A1BE08C
:103D4000030A0FE0010A2EE10101E46BE36B320E7E
:103D5000E56FE66FE76FE86FE96FEA6FEB6FEC6FA7
:103D600021D003C1E4F10101E45102E1000E01D0D0
:103D7000010EE36F17D003C1E5F104C1E6F105C1FF
:103D8000E7F106C1E8F107C1E9F108C1EAF109C1AB
:103D9000EBF10AC1ECF106D00351050DF3CFEDF1C3
:103DA000F4CFEEF10101100E006F1200D9CFE6FF43
:103DB000E1CFD9FF020EE126D00EDE6E070EDD6EDA
:103DC0000101DAA125D093908A80DB510A0DED51D3
:103DD000F324106EEE51F420116E10C0E6FFE66E73
:103DE000E9DAE552E5520101DB51106E116AD9CFD3
:103DF000E9FFDACFEAFF1050EE5E1150ED5AD9CF4D
:103E0000E9FFDACFEAFF640EEE5E000EED5A8A900B
:103E1000DAA325D093928A82DC510A0DED51F32466
:103E2000106EEE51F420116E10C0E6FFE66EC2DA9D
:103E3000E552E5520101DC51106E116AD9CFE9FF5C
:103E4000DACFEAFF1050EE5E1150ED5AD9CFE9FFFC
:103E5000DACFEAFF640EEE5E000EED5A8A92DAA522
:103E600025D093948A84DD510A0DED51F324106E10
:103E7000EE51F420116E10C0E6FFE66E9BDAE552BB
:103E8000E5520101DD51106E116AD9CFE9FFDACF99
:103E9000EAFF1050EE5E1150ED5AD9CFE9FFDACFAC
:103EA000EAFF640EEE5E000EED5A8A94DAA725D082
:103EB00093968A86DE510A0DED51F324106EEE5171
:103EC000F420116E10C0E6FFE66E74DAE552E5529A
:103ED0000101DE51106E116AD9CFE9FFDACFEAFF96
:103EE0001050EE5E1150ED5AD9CFE9FFDACFEAFF5C
:103EF000640EEE5E000EED5A8A96DAA925D09398EC
:103F00008A88DF510A0DED51F324106EEE51F42032
:103F1000116E10C0E6FFE66E4DDAE552E552010182
:103F2000DF51106E116AD9CFE9FFDACFEAFF1050E6
:103F3000EE5E1150ED5AD9CFE9FFDACFEAFF640EF9
:103F4000EE5E000EED5A8A98DAAB25D0939A8A8AF3
:103F5000E0510A0DED51F324106EEE51F420116E74
:103F600010C0E6FFE66E26DAE552E5520101E051A7
:103F7000106E116AD9CFE9FFDACFEAFF1050EE5E7A
:103F80001150ED5AD9CFE9FFDACFEAFF640EEE5EA9
:103F9000000EED5A8A9ADAAD25D0939C8A8CE151B5
:103FA0000A0DED51F324106EEE51F420116E10C085
:103FB000E6FFE66EFFD9E552E5520101E151106ED0
:103FC000116AD9CFE9FFDACFEAFF1050EE5E115047
:103FD000ED5AD9CFE9FFDACFEAFF640EEE5E000EAC
:103FE000ED5A8A9CDAAF25D0939E8A8EE2510A0D53
:103FF000ED51F324106EEE51F420116E10C0E6FF67
:10400000E66ED8D9E552E5520101E251106E116A0F
:10401000D9CFE9FFDACFEAFF1050EE5E1150ED5A2A
:10402000D9CFE9FFDACFEAFF640EEE5E000EED5A5B
:104030008A9ED9CFE9FFDACFEAFF000ED880EE548E
:10404000000EED5414E2DECF10F0DDCF11F00A0EB9
:104050001102F3CF11F01002F3CF10F0F45011263B
:10406000F3CFE6FF11C0E6FFA5D9E552E552020EF7
:10407000E15C02E2E16AE552E16EE552E7CFD9FF89
:104080001200D9CFE6FFE1CFD9FF020EE126E20E02
:10409000DE6E040EDD6E0101E4A125D094908B80CC
:1040A000E5510A0DED51F324106EEE51F420116E1E
:1040B00010C0E6FFE66E7ED9E552E5520101E551FA
:1040C000106E116AD9CFE9FFDACFEAFF1050EE5E29
:1040D0001150ED5AD9CFE9FFDACFEAFF640EEE5E58
:1040E000000EED5A8B90E4A325D094928B82E6517A
:1040F0000A0DED51F324106EEE51F420116E10C034
:10410000E6FFE66E57D9E552E5520101E651106E21
:10411000116AD9CFE9FFDACFEAFF1050EE5E1150F5
:10412000ED5AD9CFE9FFDACFEAFF640EEE5E000E5A
:10413000ED5A8B92E4A525D094948B84E7510A0D17
:10414000ED51F324106EEE51F420116E10C0E6FF15
:10415000E66E30D9E552E5520101E751106E116A61
:10416000D9CFE9FFDACFEAFF1050EE5E1150ED5AD9
:10417000D9CFE9FFDACFEAFF640EEE5E000EED5A0A
:104180008B94E4AD25D0949C8B8CEB510A0DED51B2
:10419000F324106EEE51F420116E10C0E6FFE66EAF
:1041A00009D9E552E5520101EB51106E116AD9CFE0
:1041B000E9FFDACFEAFF1050EE5E1150ED5AD9CF89
:1041C000E9FFDACFEAFF640EEE5E000EED5A8B9C3B
:1041D000E4AF25D0949E8B8EEC510A0DED51F32463
:1041E000106EEE51F420116E10C0E6FFE66EE2D8BC
:1041F000E552E5520101EC51106E116AD9CFE9FF89
:10420000DACFEAFF1050EE5E1150ED5AD9CFE9FF38
:10421000DACFEAFF640EEE5E000EED5A8B9ED9CF28
:10422000E9FFDACFEAFF000ED880EE54000EED541D
:1042300014E2DECF10F0DDCF11F00A0E1102F3CF41
:1042400011F01002F3CF10F0F4501126F3CFE6FF77
:1042500011C0E6FFAFD8E552E552020EE15C02E282
:10426000E16AE552E16EE552E7CFD9FF1200D9CFFE
:10427000E6FFE1CFD9FF020EE12601010251040A57
:1042800033E0070A27E0010A19E0030A07E0010A00
:1042900032E191EC2BF00101CD892DD03F0EE66E7D
:1042A00064EC2AF0E552000EE66EE66A48EC2AF06D
:1042B000E552E55292880101CD991DD0EEEC29F02E
:1042C000F3CFDEFFF4CFDDFFDFCF03F1010EDBCF55
:1042D00004F111D003C1DFFF010E04C1DBFFDECF0B
:1042E000E6FFDDCFE6FF03D0000EE66EE66A48EC9F
:1042F0002AF0E552E5520101100E006F020EE15C5A
:1043000002E2E16AE552E16EE552E7CFD9FF120021
:10431000D9CFE6FFE1CFD9FF020EE126010102511C
:10432000040A34E0070A28E0010A1AE0030A07E059
:10433000010A33E18EEC2BF00101CF812ED0070E64
:10434000E66E8FEC29F0E552CD96000EE66EE66A39
:104350002CEC2AF0E552E55294800101CF911DD05A
:10436000CFEC29F0F3CFDEFFF4CFDDFFDFCF03F199
:10437000010EDBCF04F111D003C1DFFF010E04C138
:10438000DBFFDECFE6FFDDCFE6FF03D0000EE66EFB
:10439000E66A2CEC2AF0E552E5520101100E006F9E
:1043A000020EE15C02E2E16AE552E16EE552E7CF1E
:1043B000D9FF1200D9CFE6FFE1CFD9FFE652FF0EB9
:1043C000E76EFD0EDBCF10F0E7501016116A1050AB
:1043D000DF6EDF50000805E2DFCFE6FF7CEC2BF05C
:1043E000E552FD0EDBCF10F0FE0EDBCF11F011C059
:1043F00010F0116A1050DF6EDF50000832E2DFCF9C
:10440000E6FF41EC2BF0E552DFCFE6FF41EC2BF06D
:10441000E552DFCFE6FF41EC2BF0E552DFCFE6FFC0
:104420007CEC2BF0E552DFCFE6FF7CEC2BF0E55285
:10443000DFCFE6FF7CEC2BF0E552DFCFE6FF7CEC34
:104440002BF0E552DFCFE6FF7CEC2BF0E552DFCF1F
:10445000E6FF7CEC2BF0E552DFCFE6FF7CEC2BF0A7
:10446000E552E552E552E7CFD9FF1200D9CFE6FF7A
:10447000E1CFD9FFE150FD0FE96EFF0EDA20EA6EC1
:10448000000ED880EE54000EED5412E2FD0EDBCF8C
:10449000E6FFFCEC2AF0E552FD0EDBCFE6FF41EC37
:1044A0002BF0E552FD0EDBCFE6FF41EC2BF0E552A1
:1044B000E552E7CFD9FF1200D9CFE6FFE1CFD9FF10
:1044C000030EE1260101440E016F3F0E006F040E42
:1044D000DF6E0251E66ED950010FE96EDACFEAFFC6
:1044E000E552E750EE6EED6A010EDBCF10F0020EE2
:1044F000DBCF11F002510425136AE850105C135011
:10450000115814E2A69E010EDB50A96EA680DF5062
:10451000EA6A010FE96E010EEA22A8CFEFFFDF2A57
:10452000010EDB2A020EE0E3DB2ADED7030EE15C9C
:1045300002E2E16AE552E16EE552E7CFD9FF1200EF
:10454000D9CFE6FFE1CFD9FF030EE1260101010E2D
:10455000006F450E016F040EDF6E0251E66ED950FA
:10456000010FE96EDACFEAFFE552E750EE6EED6A31
:10457000010EDBCF10F0020EDBCF11F00101025172
:104580000425136AE850105C135011581CE2A69ED3
:10459000A684010EDB50A96EDF50EA6A010FE96EB6
:1045A000010EEA22EF50A86E550EA76EAA0EA76E56
:1045B000A682A1A8FED7A198DF2A010EDB2A020E4F
:1045C000D7E3DB2AD5D7030EE15C02E2E16AE552CC
:1045D000E16EE552E7CFD9FF1200C282C2B2FED728
:1045E00012009494780ECB6E0C0EBD6EBE6E040E4F
:1045F000CA6E12006C500CE16896040100513C0B2D
:10460000E842E8420D0802E10AD8010C1ED8010C6C
:10461000040E6C5C03E1689627D8010C000CD9CF1E
:10462000E6FFE1CFD9FFE652040104BF046B0001AD
:10463000686B606B616B666B676B9DEC24F0E8D810
:10464000E552E552E7CFD9FF1200020E0001605D8E
:1046500009E1A1D8040100BD02D0C80E01D0880E26
:10466000006F12004DEF24F0040E0101F95D09E125
:104670001AC46EFF6E50000802E2050E01D0030E50
:10468000F96F0001600510E111D8020E0001685DAC
:1046900003E10401840E06D0040104BD02D0C80E5B
:1046A00001D0880E046F12004DEF24F0D9CFE6FF41
:1046B000E1CFD9FF020EE1260001080E665D000E73
:1046C00067590DE266C0DEFF67C0DDFF685102E199
:1046D000010E03D0680506E1020E686F03D0080ED4
:1046E000DE6EDD6A040104930491010EDB500413B5
:1046F000DFCF05F4000EDB500001665F010EDB50DA
:10470000675B200E646F040E656F0101FAA31DD074
:10471000D9CFE9FFDACFEAFFEE50ED1032E062C008
:10472000F6FF63C0F7FF0800F55064C0E9FF65C0FD
:10473000EAFFEF6E0001642B000E6523622B6323FA
:10474000DF06010EE5E2DB06E3D7D9CFE9FFDACFDA
:10475000EAFFEE50ED1015E062C0E9FF63C0EAFF2A
:10476000EF5064C0E9FF65C0EAFFEF6E0001642B03
:10477000000E6523622B6323DF06010EE6E2DB06F3
:10478000E4D7020EE15C02E2E16AE552E16EE55235
:10479000E7CFD9FF1200D9CFE6FFE1CFD9FF020E54
:1047A000E126030E04010015E76E010EE7CFDBFFE3
:1047B00001C4DFFFDE5000016627DD506723200EB5
:1047C000626F040E636FD9CFE9FFDACFEAFFEE50D4
:1047D000ED1014E062C0E9FF63C0EAFFEF5064C06F
:1047E000E9FF65C0EAFFEF6E642B000E6523622BC4
:1047F0006323DF06010EE7E2DB06E5D7020EE15C8C
:1048000002E2E16AE552E16EE552E7CFD9FF12001C
:104810006D98000161510BE10401080E016F180E43
:10482000026F040E036F840E006F040123D0040195
:1048300018AF22D00001665104011E5D00016751CE
:1048400004011F5904E21EC466F01FC467F02EDF86
:104850000001010E606F0401080E016F180E026F57
:10486000040E036F800E006F0401200E066F040E0D
:10487000076FC80E046F12000001020E606F040182
:10488000056BC80E046F0401080E016F200E026F45
:10489000040E036FC80E006F1200D9CFE6FFE1CF00
:1048A000D9FFE652020E0001605D35E16D50100B3C
:1048B00032E004010151106E116A080E10182BE14C
:1048C000115029E100513C0BE842E8420D0823E178
:1048D0000051800B20E1180E026F040E036FDF6A97
:1048E000DF50106E116A080E105C000E115820E2A5
:1048F000DF50EA6A200FE96E040EEA22EF50E66EFE
:10490000DF50EA6A180FE96E040EEA22E552E7501A
:10491000EF6EDF2AE5D70001606B0401080E016F1E
:10492000180E026F040E036F8C0E006F0401046BEF
:10493000E552E552E7CFD9FF120004011851600B90
:10494000E842E842E842E842E842000901E0120099
:104950001951070A4CE00B0A4AE0070A3BE0010A3A
:1049600027E00B0A23E0020A21E0030A1DE0080AFF
:1049700012E0010A0EE00F0A0AE0030A01E0120049
:104980000001010E616F0101040EF96F1200F8EFD2
:1049900024F04FEF25F00001010E616F0001FB0EC6
:1049A000626F010E636F10D076EF25F0C1EF25F036
:1049B0000001010E616F04011C510001626F636B05
:1049C000FC0E6227010E63230101FA930001010E20
:1049D000666F12000001010E616F04011C51EA6A4A
:1049E000FC0FE96E010EEA221AC4EFFF120012005A
:1049F000800E0401185D52E11B51030A30E0010AE8
:104A00000CE0030A49E10001010E616F0001DE0EB6
:104A1000626F4E0E636F120E3CD00001010E616F8B
:104A200004011A51F66EF76AD890F636F736740E0E
:104A3000F6264F0EF7220900F5CF62F00A00F5CFF7
:104A400063F0020E0001F76A6225F66E6351F722E9
:104A50000900F5CF66F00A00F5CF67F01DD0000120
:104A6000010E616F04011A51F66EF76AD890F6369E
:104A7000F736780EF6264F0EF7220900F5CF62F0D2
:104A80000A00F5CF63F062C0F6FF63C0F7FF0800CD
:104A9000F5500001666F676B0101FA831200000197
:104AA000010E616F0F0EE66E710EE66E0F0EE66E72
:104AB000CCEC26F0E552E552E552010EE66EFC0E16
:104AC000E66E010EE66ECCEC26F0E552E552E552BC
:104AD0001AC4FBF104011A5104E10101050EF96F3A
:104AE00012000101060EF96FE1EF26F00401206BC0
:104AF000216B040118511F0B020A13E0030A0DE099
:104B0000010A31E10001010E616F04012081010100
:104B1000FAA129D00401208326D00001010E616F83
:104B200022D00001010E616F04011C510F0B080D12
:104B3000F350116A000F106E040E11221C51800BED
:104B400001E0010E040DF35000011024646F000E0B
:104B50001120656F64C0E9FFEA6EEF50040B03E0BB
:104B60000401010E206F000161050AE10001200E21
:104B7000626F040E636F0101FA930001020E666F0B
:104B8000120004011A0510E118511F0B00090CE175
:104B90000001010E616F030E0401195D03E10101C3
:104BA000FA8102D00101FA9104011A5136E118513B
:104BB0001F0B020832E11C510F0B00092EE000010F
:104BC000010E616F04011C510F0B080DF350116AA7
:104BD000000F106E040E11221C51800B01E0010E1B
:104BE000040DF35000011024646F000E1120656F56
:104BF000030E0401195D02E1840E03D01CAF07D03F
:104C0000400E64C0E9FF65C0EAFFEF6E1200880E37
:104C100064C0E9FF65C0EAFFEF6E12006DA60CD814
:104C20000101F90508E16DBA06D0686A696A698010
:104C30006988020EF96F12006D6A696A6D8601015A
:104C4000010EF96F12006D6A696A0101F96B1200B9
:104C500023EF26F00101F95101E112006850040B25
:104C600004E06950040B01E042D86DB212006850B4
:104C7000010B04E06950010B01E066D86850100B8D
:104C800004E06950100B01E02ED86850400B04E09E
:104C90006950400B01E044D86850200B04E0695093
:104CA000200B01E03FD86850020B04E06950020B72
:104CB00001E048D8030E0101F95D01E21200010193
:104CC000FD6B040EFD5D0EE26850080B0BE06950B1
:104CD000080B08E0FAEC22F0000901E168960101F6
:104CE000FD2BEFD71200698468986D8212006D92D7
:104CF000699468A402D06894FCD712000101FAA15B
:104D00000ED06D926D840101080EFE6F070EFF6FCD
:104D1000FE07000EFF5BFE51FF11FAE16D941200D9
:104D2000689C120070A00CD0800E0401005D07E1A9
:104D3000840E0401045D03E104018C0E006F709089
:104D4000689A12006A6A12006A6A686A9F0E6B6E3D
:104D50007B0E696E6E6A0F0EE66E710EE66E0F0EBA
:104D6000E66E1AD8E552E552E552160E706E68A648
:104D700008D068960000000000000000000000005D
:104D8000F6D76D984DEC24F00101FA910101FB6B0F
:104D90000101030EF96F1200D9CFE6FFE1CFD9FF71
:104DA000FD0EDBCFE9FFFE0EDBCFEAFFFC0EDB5092
:104DB00004E0EE6AFC0EDB06F9D7E552E7CFD9FF37
:104DC00012000001696B1E0E716E0401400E096F26
:104DD000280E0A6F040E0B6F880E086F0401680E10
:104DE0000E6F040E0F6F400E0C6F1200D9CFE6FF4E
:104DF000E1CFD9FFE652FC0EDB50400805E2400E41
:104E0000F36EFC0EF3CFDBFFDF6AFC0EDB50DF5CE2
:104E100019E2DF50E76EFD0EDBCFE9FFFE0EDBCFC0
:104E2000EAFFE750E926000EEA22EF50E66EDF5077
:104E3000EA6A680FE96E040EEA22E552E750EF6E67
:104E4000DF2AE3D7FC0EDBCF0DF4400E04010C1774
:104E50000C7D880E0C13E552E552E7CFD9FF120006
:104E6000D9CFE6FFE1CFD9FF0001696B040108BF8C
:104E700030D0FC0EDBCF10F00951D880105403E283
:104E8000FC0E09C4DBFF0001696BFC0EDB50695DA1
:104E900019E26951EA6A280FE96E040EEA22EF501E
:104EA000E66E6951E76EFD0EDBCFE9FFFE0EDBCF4C
:104EB000EAFFE750E926000EEA22E552E750EF6EDE
:104EC000692BE3D70401400E096F0817087D880E8F
:104ED000081300016951E552E7CFD9FF1200120112
:104EE000000200000008D8040BFF010001020001CD
:104EF00009022000010100C0320904000002000084
:104F00000000070501024000000705810240000083
:104F1000040309042A037300700072007500740012
:104F2000200028007700770077002E0073007000C3
:104F30007200750074002E006400650029003603BD
:104F4000550053004200340061006C006C002D00DD
:104F50004D00430044002000390020002800730069
:104F600070007200750074002000320030003100C3
:104F700032002900F04EF04E104F144F3E4F2A0ED3
:104F8000F66E080EF76E000EF86E01010900F5507E
:104F9000F46F0900F550F56F03E1F46701D03DD0DF
:104FA0000900F550EF6F0900F550F06F0900F5505A
:104FB000F16F09000900F550E96E0900F550EA6E3D
:104FC000090009000900F550F26F0900F550F36F70
:104FD00009000900F6CFF6F1F7CFF7F1F8CFF8F1B5
:104FE000EFC1F6FFF0C1F7FFF1C1F8FF0101F25385
:104FF00002E1F35307E00900F550EE6EF207F8E224
:10500000F307F9D7F6C1F6FFF7C1F7FFF8C1F8FFCC
:105010000101F407000EF55BBFD71200D9CFE6FF00
:10502000DACFE6FFE1CFD9FFE2CFDAFFAC6AAB6AB5
:10503000FD0EDBB0AC88DBA202D0AC8CAB8CDBB459
:10504000AC8EDBA602D0AB8801D0AB8ADBB8AC84D7
:105050009E98DBBAAB86DBAC02D09D8A01D09D9ACC
:105060009E9ADBAE02D09D8801D09D98FB0EDB504E
:10507000AF6EFB0EFC0EDBCF11F011C010F0116A09
:105080001050B06EAC8AAB8E949C948EAC50100BCA
:1050900004E0AC50800B01E1948CE552E5CFDAFFDF
:1050A000E7CFD9FF1200D9CFE6FFDACFE6FFE1CF95
:1050B000D9FFE2CFDAFFE652E652E652E652F8CFE7
:1050C00002F0F6CF03F00C0EBA6E050EF66EF76A1C
:1050D000300EF86E0800F550010B03E0010EDB689E
:1050E00002D0010EDB6A010EDB5002E0949201D087
:1050F0009396CA94FD0EDB50CB6ECA8402C0F8FFB3
:1051000003C0F6FF040EE15C02E2E16AE552E16EE3
:10511000E552E5CFDAFFE7CFD9FF1200D9CFE6FF9E
:10512000DACFE6FFE1CFD9FFE2CFDAFFFD0EDB50A9
:10513000C96EC6AE02D0FF0E24D00F0EC6140808EA
:105140000FE00F0EC6140B080BE0C6889EA6FED714
:10515000C750040B03E1C750010B10E0000E11D043
:105160000F0EC614080804E00F0EC6140B0809E160
:10517000C7B0FED787EC2BF0C5AC02D0FE0E01D035
:10518000000EE552E5CFDAFFE7CFD9FF1200045059
:105190000902F3CF00F0F4CF01F00A02F350012628
:1051A000000EF420026E04500B02F3500226000E93
:1051B000F420036E04500C02F3500326055009023C
:1051C000F3500126F4500222000E032205500A0279
:1051D000F3500226F450032205500B02F35003262D
:1051E00006500902F3500226F450032206500A0228
:1051F000F350032607500902F35003261200D9CFBB
:10520000E6FFDACFE6FFE1CFD9FFE2CFDAFF3F0ECC
:10521000C716C66AFD0EDB50C612FB0EDB50C71266
:10522000FC0EDB50030A09E0010A04E0020A06E171
:10523000C78C04D0C78CC68801D0C688FD0EDB5051
:10524000050A03E0010A03E1928A938201D0939256
:105250009380949EC68AE552E5CFDAFFE7CFD9FF67
:105260001200D9CFE6FFDACFE6FFE1CFD9FFE2CFD8
:10527000DAFFE652E652FC0EDBCF10F0FD0EDBCF7C
:1052800011F0060ED89010361136E804FBE110C07C
:10529000DEFF11C0DDFF010EDB50BB6EDF50E840CA
:1052A000E8403F0B300B106ECF0EBA141010BA6EE0
:1052B000E552E552E552E5CFDAFFE7CFD9FF12001C
:1052C000D9CFE6FFDACFE6FFE1CFD9FFE2CFDAFFB1
:1052D000E652E652FC0EDBCF10F0FD0EDBCF11F0F4
:1052E000060ED89010361136E804FBE110C0DEFF40
:1052F00011C0DDFF010EDB50BE6EDF50E840E8401C
:105300003F0B300B106ECF0EBD141010BD6EE5526A
:10531000E552E552E5CFDAFFE7CFD9FF1200D9CF4A
:10532000E6FFDACFE6FFE1CFD9FFE2CFDAFFFD0EED
:10533000DB50360BB16EB36AB26AA192FD0EDBAEE2
:1053400002D0A08201D0A092DBA002D0B18E01D009
:10535000B19EB180E552E5CFDAFFE7CFD9FF120069
:10536000D9CFE6FFDACFE6FFE1CFD9FFE2CFDAFF10
:10537000E652F20E00016A17ABAC03D06A91ABB0F3
:105380006A81ABB46A85ABB26A87AE50DF6EDF501C
:10539000E552E552E5CFDAFFE7CFD9FF1200D9CFCA
:1053A000E6FFDACFE6FFE1CFD9FFE2CFDAFFE65240
:1053B000E652B250DF6E010EB3CFDBFFDECF10F04E
:1053C000DDCF11F010C0F3FF11C0F4FFE552E5523C
:1053D000E552E5CFDAFFE7CFD9FF1200D9CFE6FFDC
:1053E000DACFE6FFE1CFD9FFE2CFDAFFE652E652AD
:1053F000D650DF6E010ED7CFDBFFDECF10F0DDCF52
:1054000011F010C0F3FF11C0F4FFE552E552E55270
:10541000E5CFDAFFE7CFD9FF1200D9CFE6FFDACF29
:10542000E6FFE1CFD9FFE2CFDAFFC688FD0EDB5001
:10543000C96EC7A0FED7FC0EDB50C96EC7A0FED751
:10544000C698C96AC7A0FED7C688C950E552E5CF3D
:10545000DAFFE7CFD9FF1200D9CFE6FFDACFE6FFB8
:10546000E1CFD9FFE2CFDAFFE652E652FC0EDBCF06
:10547000DEFFDBCFDDFF010EDB50B36EDF50B26E1F
:10548000E552E552E552E5CFDAFFE7CFD9FF12004A
:10549000D9CFE6FFDACFE6FFE1CFD9FFE2CFDAFFDF
:1054A000E652E652FC0EDBCFDEFFDBCFDDFF010E66
:1054B000DB50D76EDF50D66EE552E552E552E5CFB0
:1054C000DAFFE7CFD9FF1200D9CFE6FFDACFE6FF48
:1054D000E1CFD9FFE2CFDAFFFD0EDB507F0BD56EB7
:1054E000D76AD66AF294FD0EDBAE02D0F28A01D002
:1054F000F29AD58EE552E5CFDAFFE7CFD9FF120059
:10550000D9CFE6FFDACFE6FFE1CFD9FFE2CFDAFF6E
:10551000FD0EDB50FB0BCA6ECC6A9E92FD0EDBAE1D
:1055200002D09D8201D09D92CA84E552E5CFDAFF78
:10553000E7CFD9FF1200D9CFE6FFDACFE6FFE1CF00
:10554000D9FFE2CFDAFFC688FD0EDB50C96EC6AECA
:1055500002D0FF0E03D0C7A0FED7000EE552E5CF64
:10556000DAFFE7CFD9FF1200D9CFE6FFDACFE6FFA7
:10557000E1CFD9FFE2CFDAFF0C0EBD129494CA94AA
:10558000FD0EDB50CB6ECA84E552E5CFDAFFE7CFE4
:10559000D9FF120094941200D9CFE6FFDACFE6FFCC
:1055A000E1CFD9FFE2CFDAFF3F0EC716C66AFD0E84
:1055B000DB50C612949E93929380C68AE552E5CF43
:1055C000DAFFE7CFD9FF120004D80FD820EC05F09E
:1055D000FCD70F0EC112140E6F6E0101F96B0101A1
:1055E000FA6B0101FB6B1CEF04F00EEC26F06FBEB2
:1055F00002D02AEC26F01200FF0EE350156EEF0EDB
:1056000001D0F30EE76EE72E03EF2BF00C0E146EB5
:10561000E76AE72E09EF2BF0142E08EF2BF0152E7A
:1056200001EF2BF01200D9CFE6FFDACFE6FFE1CF92
:10563000D9FFE2CFDAFFACAC04D0AC9000016AB382
:10564000AC80FD0EDB50AD6EE552E5CFDAFFE7CF63
:10565000D9FF1200D9CFE6FFDACFE6FFE1CFD9FFBD
:10566000E2CFDAFFE652C950DF6E9E96C96A9EA667
:10567000FED7C950E552E552E5CFDAFFE7CFD9FFB3
:105680001200FF0EE350156E480E01D04C0EE76E6F
:10569000E72EFED7E76AE72EFED7152EF7D70000D4
:1056A0001200000EF36E00EE00F0080E01D812009A
:1056B000EA6002D0EE6AFCD7F350E9601200EE6AAD
:1056C000FCD713EE00F023EE00F0F86A0F9CBFEC5D
:1056D00027F098EC2BF0E4EC2AF0FBD712000F0E29
:1056E000C614080804E00F0EC6140B0801E1C586B5
:1056F000C7A0FED7C9501200FF0EE350E84E1200BB
:10570000000000D000D000D0E82EFAD712001F0E03
:10571000C514FDE1C750040BFAE11200B190A0924C
:105720001200D59EF29A1200BA6A1200BD6A1200E7
:1057300012000210007FFFC700000000000064009C
:105740000000003232323232323232000032323233
:085750003232323232E803FF6D
:020000040030CA
:0E000000240E381E008181000FC00FA00F409B
:00000001FF
